:020000040000FA
:040000001920572943
:040004000034003490
:08000800F000030EF100831269
:10001000031383130408F2000A08F3008C183E202F
:1000200073088A0072088400710E8300F00E700E4F
:020030000900C5
:0E00320083160130930083120030F400850025
:1000400083161F3085008312831687308100831248
:1000500083165F309F0083120130D6009F000C3062
:100060009500FF30831692008312003092004030DA
:100070008B00831602308C00831208008C10411014
:10008000050840060839031D411455204508930012
:1000900095121512C41B9516441B15160800C101B4
:1000A000C501C401C301C201080041196228C11978
:1000B0008428411ABB28C11AC8285E28411C0800A0
:1000C0004115080046080318460FC20747080318E1
:1000D000470FC30748080318480FC4074908031807
:1000E000490FC50703187728411C81280800FF30F5
:1000F000C200C300C400C500411C81284111C115C4
:1001000008004111C11608004A08031C4A0FC20228
:100110004B08031C4B0FC3024C08031C4C0FC402BA
:100120004D08031C4D0FC502031CAB284E08031CD1
:100130004E0F42024F08031C4F0F43025008031C8E
:10014000500F44025108031C510F4502031CAB28F9
:10015000411CB82808004E08C2004F08C3005008D0
:10016000C4005108C500411CB828C111411608003F
:10017000C111C11608004E08C2004F08C300500844
:10018000C4005108C500411808004112C1160800FA
:100190005208031C520FC2025308031C530FC30220
:1001A0005408031C540FC4025508031C550FC50204
:1001B000031CDD284118E5280800C201C301C40161
:1001C000C501C1124118E5280800C11241150800F7
:1001D000D7019F14EF20EF20EF20EF2008009F1899
:1001E000EF281E08D8000430D607561256089F0084
:1001F000023057020319FE281D2103295808DE008A
:10020000DD01DC01DB010310570D84000310840DB8
:1002100046308407C1188B135B088000840A5C0891
:100220008000840A5D088000840A5E088000C1188E
:100230008B17D70A57119F140800580D1E39DA0082
:100240000310DA0DC030DA0703308A00580E0F3978
:10025000D8005B308400D8193C2955218000DA0A87
:10026000840A55218000DA0A840A55218000DA0ABE
:10027000840A552180004A29DA0A55218000DA0AC9
:10028000840A55218000DA0A840A55218000840AF4
:100290008001D811D808031908000310DE0CDD0C0A
:1002A000DC0CDB0CD80B4D2908005A0882004F20CB
:1002B000E8200508C000C11412158B17EF205E2935
:10078000A5349B34C43420346234F53460341F34CF
:10079000303463340C341E3465344134C6341C3474
:1007A0004D34F3348D341B34D334E23462341A3490
:1007B0004334803444341934FF34413432341834EF
:1007C0003F34A4342B341734D23428343034163424
:1007D000DE3456343F341534AC34BA34583414341F
:1007E0006A34E5347B341334FC346C34A83412346A
:1007F000C334EB34DD3411346F3400341C34113421
:084000000000010003000000B4
:02400E00C43FAD
:00000001FF
